:020000040000FA
:100000003028000000000000F200030E8301F5001C
:100010000A08F4008A010408F300831203138C1EFB
:1000200027281A08981C18281A08181218160D28BC
:1000300083160313F600A10AE3302102031D2228D0
:10004000A230A10021088400760880000D287308E2
:10005000840074088A00750E8300F20E720E090087
:100060008301831603132730810000308C00003099
:100070008D00EF30850000308600B0308700003002
:100080009F0083120313003085000030860000308B
:100090008700C0308B00003090008C0197019D01DB
:1000A000203084008001840A6D300402031C522831
:1000B0005B24BC24782083160313A230A100A00087
:1000C0008C1683120313C52007142830A4005C305B
:1000D000A5008F30A6000230A7009320A6201A2189
:1000E000031C6F28A0008F302002031D6F283429C5
:1000F0008312031307168316031307121430990093
:10010000181598168312031318169817071208006B
:1001100007128C1E89281A080800871A8D280C1EC1
:100120008F289900080007100030A900B82000307F
:10013000A900B8200030A900B8200030A900B820DC
:100140005830A900B8208715871108000330A9008E
:10015000B8202708A900B8202608A900B82025083B
:10016000A900B8202408A900B82087158711080025
:100170000830A1000310A90D03180715031C07116F
:1001800087148710A10BBB280800FF30AB0011219A
:10019000AB0BC72806100611FF30AB001121AB0BCB
:1001A000CE280830AB001030A000A00C0821AB0B0B
:1001B000D5280830AB009830A000A00C0821AB0B6C
:1001C000DD280630AB00D030A000A00C0821AB0B1E
:1001D000E52802210830AB00E830A000A00C08217F
:1001E000AB0BEE280830AB000E30A000A00C0821AD
:1001F000AB0BF6280630AB00F030A000A00C0821B5
:10020000AB0BFE2811210614112106101121080044
:1002100003188614031C86100615112106111121DE
:1002200008000230EA004A30E900E90B1529EA0B20
:1002300015290800831603132108200283120313D3
:10024000031D24290310080083160313A00AE330BA
:100250002002031D2D29A230A000200884000008E0
:100260008312031303140800D9211A21031C352912
:10027000E800603068020318D9214F3084004E082E
:10028000840768088000CE0A4F08773A031D4F297B
:100290004E08163A031D4F292A14DF22D7294F088A
:1002A000663A031D59294E080A3A031D59290B24A1
:1002B000D7294F08783A031D64294E08163A031DC2
:1002C00064292A10DF22D7294F086D3A031D6E29B1
:1002D0004E08013A031D6E29D523D7294F08653AE8
:1002E000031D78294E080D3A031D78291B24D729B0
:1002F0004F08763A031D82294E08013A031D8229D0
:100300005724D7294F08723A031D8C294E08023A08
:10031000031D8C295C24D7294F08613A031D9729B6
:100320004E08193A031D97292A10DD22D7294F08B4
:10033000623A031DA2294E08193A031DA2292A1464
:10034000DD22D7294F08733A031DAC294E08013A24
:10035000031DAC294724D7294F086F3A031DB6293E
:100360004E08023A031DB6295A24D7294F08633A8A
:10037000031DC1294E081B3A031DC1292A1037232A
:10038000D7294F08643A031DCC294E081B3A031D98
:10039000CC292A143723D7294F086E3A031DD629B2
:1003A0004E08013A031DD629E623D7293529D9213C
:1003B0006F2863220800D201D301D401D501D601F0
:1003C000D701CE01CF01D001D1010800DB214808BF
:1003D00084000008CE00840A0008CF00840A0008C8
:1003E000D000840A0008D100840A0008D200283016
:1003F000AB000310D20CD10CD00CCF0CCE0CD70C10
:10040000D60CD50CD40CD30C4E3084000530AC0087
:10041000801F0C2A30308002801D102A0330800299
:10042000840AAC0B082AAB0BF9294808840053084E
:100430008000840A54088000840A55088000840AD9
:1004400056088000840A5708800008002E08D8004B
:100450002F08D9003008DA003108DB003208DC0050
:100460002030D6005830C8006030C900CF010310DA
:10047000D50CD40CD30CD20C031C572A0830D00056
:10048000480884000008CE00490884004F08CF01C6
:100490008007031C4D2A0130CF004E088007031C43
:1004A000532A0130CF00C80AC90AD00B402A0310D2
:1004B000D80DD90DDA0DDB0DDC0DDD0DDE0DDF0DF8
:1004C000D60B322A08004E308400800167300402C7
:1004D00003196C2A840A652A080050080F39B800ED
:1004E000510EF039B70052080F39B704530EF039E6
:1004F000B60054080F39B604550EF039B500560849
:100500000F39B504570EF039B40058080F39B40448
:100510000800BD01590EF039BC005A080F39BC045F
:100520005B0EF039BB005C080F39BB045D0EF0397F
:10053000BA005E080F39BA045F0EF039B9006008DE
:100540000F39B9040800C001C101C201610EF039C0
:10055000BF0062080F39BF04630EF039BE006408A3
:100560000F39BE040800C401C501C601C7016508F2
:100570000F39C404660EF039C30067080F39C3048D
:100580000800FB01FC01FD01FE01FF01680EF039CE
:10059000FB0069080F39FB0408004308EA0044081F
:1005A000EB000F30E900E90BD32AEA0BD12AEB0864
:1005B0000319DC2AEB03D12A0800B322E12AC30184
:1005C000C4018316031380309F00831203136D222E
:1005D0008922A3223430C800E6213930C800E62140
:1005E0003E30C800E6214330C800E62163223508CA
:1005F000D3003408D2003608D4003708D5002622AC
:100600007024C308031D082BC408031D082B092BE5
:10061000CD227D2422088F2023088F207B242208CE
:100620008F2023088F203908B4073A0803183A0F9F
:10063000B5073B0803183B0FB6073C0803183C0FEF
:10064000B70763223508D3003408D2003608D40037
:100650003708D50026227024BE033E0A0319BF03C3
:10066000BE08031D012BBF08031D012B08008316C4
:10067000031380309F0083120313C122B3226D2223
:100680008922A3223430C800E6213930C800E6218F
:100690003E30C800E6214330C800E6217B30C80068
:1006A000E62163223508D3003408D2003608D4008E
:1006B0003708D50026227024D724C7237808FA00EB
:1006C0007708F9007808E7007708E600DF24323081
:1006D000C000E001C00803196F2BC003DB244408ED
:1006E000D9004308D800F224C7237808E30077082C
:1006F000E2007808E7007708E6007908E2027A0865
:10070000031C7A0FE302E31F8A2BE209E309E20AE2
:100710000319E30A63087C020318972BE00A0530EB
:10072000C000DF246708FA006608F900742B670828
:10073000FA006608F90060088F2000308F206608F4
:100740008F2067088F203908B4073A0803183A0F3A
:10075000B5073B0803183B0FB6073C0803183C0FCE
:10076000B70763223508D3003408D2003608D40016
:100770003708D50026227024BE033E0A0319BF03A2
:10078000BE08031D692BBF08031D692B080020301C
:10079000AB00F701F8017B242208F70723080318B0
:1007A000230FF807AB0BCB2B080083160313803005
:1007B0009F00831203137F2422088F2023088F2099
:1007C0007B2422088F2023088F2008008316031320
:1007D00080309F0083120313F701F801F901FA0139
:1007E0002030AB007F242208F70723080318230FCB
:1007F000F8077B242208F90723080318230FFA07B8
:10080000AB0BF22B77088F2078088F2079088F2088
:100810007A088F2008006D223430C800E621632258
:100820003508D3003408D2003608D4003708D50084
:1008300026227024080050086824B200B20E510825
:100840006824B20452086824B100B10E5308682429
:10085000B10454086824B000B00E55086824B004F0
:1008600056086824AF00AF0E57086824AF04580834
:100870006824AE00AE0E59086824AE045A086824F5
:10088000B300B30E5B086824B304C92430280C30CD
:100890008F206C088F208316031380309F008312F3
:1008A0000313792422088F2023088F200800783032
:1008B0008F200800080008005008EC00861106127E
:1008C00086126C188615EC1806166C198616080028
:1008D000CE0041304E023030031837304E0208004F
:1008E0006508A5006408A4006608A6006708A700BC
:1008F000A6289130822CA130822C2A18812C893094
:10090000822C81309F0090241F151F19852C83167F
:1009100003131E0883120313A2001E08A30008007D
:10092000C830CE00CE0B922C0800831603178C180B
:10093000972C8312031770088D0071088C008316A2
:1009400003178C130C158B1355308D00AA308D00B6
:100950008C148B170C1183120313080083120317D6
:1009600070088D00831603178C130C148312031761
:100970000C088312031308000630AB002E308400ED
:100980000030F000AE248000840AF00AAB0BC22CC9
:1009900008000630AB000030F0002E308400000864
:1009A000F1009524840AF00AAB0BCF2C0800FA3032
:1009B000E624FA30E624FA30E624FA30E62C6430F5
:1009C000E62C0A30E62C0530E62C0130EB0007302F
:1009D000EA007C30E900E90BEB2CEA0BEB2CEB0B8B
:1009E000E72C0800D808031DF82CD9080319002D9E
:1009F000E524D803580A0319D9030319D808F22C9F
:100A000008001A30EB007730EA005530E900E90BB6
:0E0A1000072DEA0B072DEB0B072D0800000049
:02400E00723FFF
:0C42000008007B00420094000300000056
:00000001FF
